:040000008A11C32F6F
:100E0000FE00FE1F082F83137E18831700080800BA
:100E10000408FE0007308A007E08820700344F3441
:100E20005034523449344D344534203455344E34E2
:100E3000413420345434453443344C344134203428
:100E400059342034543445342034443445345634F1
:100E50004F344C34563445345234453420344534C0
:100E60004C342034453443344F340A340D34003488
:100E70004D344534203445344E34563449344134AD
:100E80005334543445343A342034253463340A34EA
:100E90000D340034F4007630F300782F7508253ACD
:100EA0000319532F542F592F75088A11B1278A110E
:100EB000782F672F730884000008F5000230F100D6
:100EC0007108F30775088A11B1278A11782F00017C
:100ED0000138F4070001FF3874078A1109278A11C5
:100EE000F500003A0319872F633A03195A2F622F2E
:100EF00000010138F4070001FF3874078A1109273F
:100F00008A11F500F508031D862F872F4E2F080044
:100F100003100030031801308B00831603130615ED
:100F200086161930990090308312031398002430EC
:100F300083160313980001308A114A278A118A11F7
:100F4000BB278A11FA007A08F800F9017808F60040
:100F50007908F7002A308A114A278A119F2F8A11AF
:100F60000028F000831203130C1EB72FB82FB22FE6
:100F7000700899000800831203138C1EC02FC12F24
:0C0F8000BB2F1A08080083018A11882F7B
:00000001FF
